:020000040000FA
:04000000CD303A289D
:08000800A000030EA100831209
:1000100005191028831601178312B23081002B288E
:1000200083160113831203140B190310A80DA90DD5
:10003000AA0DAB0DAC0DAC16FF302C02031D2B2806
:10004000FA302B02031D2B2831152A08AF0029088E
:10005000AE002808AD008B100B11210E8300A00EFE
:04006000200E090065
:0C007400203084008001840A6030040207
:10008000031C3C281230B000F92183160C30850582
:1000900087018312850187010730990000309A009B
:1000A000103083168E008312603083168F00831207
:1000B0000030831691008312C830831681008312AA
:1000C00031309000003083168C00831210308B008A
:1000D000831600309B001C141A088312BC00851D77
:1000E0001323831610309B001C141A088312BD00C2
:1000F000831630309B001C141A088312DE00F6228F
:1001000081018E018F010B118B100B108C018B174D
:10011000972031199A20B30B9528031085190314E1
:10012000B90DF0303902031955215923882864008C
:100130003210080031110130B7008B13203037071F
:1001400083169B001C141A088312A4001030370772
:1001500083169B001C141A088312A300A600023009
:10016000A6060030370783169B001C141A0883125A
:10017000A200A7000130A7068B17321CC528220950
:100180000339A200A309A409A50924082F02031D0D
:100190004F2923082E02031D4F2922082D02031D7B
:1001A0004F2901303702031DDA283D18DA283D14A3
:1001B0003E14062202303702031DE328BD18E3284F
:1001C000BD143E14152203303702031DEC283D19DF
:1001D000EC283D153E14212204303702031DF5287A
:1001E000BD19F528BD153E142D2205303702031D1B
:1001F000FE283D1AFE283D163E14392206303702ED
:10020000031D0729BD1A0729BD163E1445220730D4
:100210003702031D10293D1B10293D173E1454229F
:1002200008303702031D1929BD1B1929BD173E14BB
:10023000632209303702031D22295E1822295E1429
:100240003E146E220A303702031D2B29DE182B299B
:10025000DE143E1479220B303702031D34295E1957
:1002600034295E153E1484220C303702031D3D29CB
:10027000DE193D29DE153E148F220D303702031D95
:1002800046295E1A46295E163E149A220E3037021F
:10029000031D4F29DE1A4F29DE163E14A522B70A88
:1002A0000F303702031808009D280130B600B30054
:1002B000B400B500B70085018701B1139720B30BD7
:1002C000A529031085190314B90DF030390203195B
:1002D000CC29B40BA529013037020319B022023012
:1002E00037020319B522033037020319BA2204304A
:1002F00037020319BF22053037020319C422063022
:1003000037020319C922073037020319CE220830F9
:1003100037020319D322093037020319D8220A30D1
:1003200037020319DD220B3037020319E2220C30A9
:1003300037020319E7220D3037020319EC220E3081
:1003400037020319F1229630B400311D5E293111B4
:10035000321CAF292D090339AD00AE09AF092F1C9E
:100360005E298E018F010C1C5E290C102E1E5E2949
:100370008B1320303707BB002F08BA00E421103060
:100380003707BB002E08BA00E42100303707BB0056
:100390002D08BA00E4218B1785018701B70AB60141
:1003A0000F303702031C5E29F62208003E1C0800AD
:1003B0003E101030BB003D08BA00E4213030BB00D5
:1003C0005E08BA00E42108008B133A0883161C1556
:1003D0009A0083123B0883169B0055309D00AA307B
:1003E0009D009C1464009C18F2291C1183128B1729
:1003F0000800FF30C800CA15CB15CC15CD15CE1599
:10040000CF15D015D115D215D31508008130BD05F3
:10041000FF30DE054130C405C0000030C200C60018
:10042000BC185F14BC18DF1408008230BD05FF3013
:10043000DE058030C405C0000030C200C6005F1079
:1004400008008430BD05FF30DE054230C405C00021
:100450004030C200C6005F1008008830BD05FF3084
:10046000DE054630C405C0004030C200C6005F1043
:1004700008009030BD05FF30DE058A30C405C0009D
:100480008030C200C6005F100800A030BD05FF30FC
:10049000DE055130C405C0001030C200C600BC18D3
:1004A0005F14BC18DF140800C030BD05FF30DE0546
:1004B0007130C405C0000030C200C600BC185F1413
:1004C000BC18DF140800FF30BD05C030DE05403029
:1004D000C505C1000030C300C70008007F30BD055E
:1004E000C130DE058030C505C1000030C300C70043
:1004F00008007F30BD05C230DE054030C505C100B3
:100500004030C300C70008007F30BD05C430DE05A1
:100510004030C505C1004030C300C70008007F302F
:10052000BD05C830DE058030C505C1008030C30080
:10053000C70008007F30BD05D030DE054030C5055E
:10054000C1000030C300C70008007F30BD05E030A7
:10055000DE054030C505C1000030C300C7000800FB
:1005600010308506003087060800333085060630D7
:1005700087060800203085060030870608002130F5
:100580008506003087060800223085060030870681
:1005900008001030850602308706080010308506F6
:1005A00006308706080000308506103087060800F0
:1005B00000308506083087060800003085061030B8
:1005C00087060800003085061030870608000030D6
:1005D000850608308706080000308506103087063B
:1005E0000800003085061030870608003D180622F6
:1005F000BD1815223D192122BD192D223D1A39227F
:10060000BD1A45223D1B5422BD1B63225E186E227B
:10061000DE1879225E198422DE198F225E1A9A2250
:10062000DE1AA5220800B601B301B4013C1C1B2B45
:10063000BC01BC141D2BBC013C143C08B60064007A
:10064000212B222B232B242B252BFF30B41B8500A1
:10065000B41F8501B30B1F2BB40B1F2B0310B60C5B
:10066000B608031D1F2B0030BB003C08BA00E42174
:10067000080005125C180516DC1C8512DC188516AE
:100680005C1D05105C190514DC1D8510DC19851432
:100690005C1E87105C1A8714DC1E0711DC1A071514
:1006A0005C1F07105C1B0714DC1F8712DC1B8716FE
:1006B00008008F08031908008F0178308E00C80FDA
:1006C000872DC80A441C892B461C7A2BCA1C6B2B0D
:1006D000CA014A15972B4A1D702BCA01CA15972BC0
:1006E000CA1D752BCA014A16972B4A1E972BCA01A1
:1006F000CA14972B4A1D7F2BCA014A16972BCA1D75
:10070000842BCA014A16972B4A1E972BCA01CA147A
:10071000972BCA1C8E2BCA014A15972B4A1D932B67
:10072000CA01CA15972B4A1E972BCA014A15C41C29
:10073000BE2BC61CAF2BCB1CA02BCB014B15CC2B3F
:100740004B1DA52BCB01CB15CC2BCB1DAA2BCB0145
:100750004B16CC2B4B1ECC2BCB01CB14CC2B4B1DD7
:10076000B42BCB014B16CC2BCB1DB92BCB014B168D
:10077000CC2B4B1ECC2BCB01CB14CC2BCB1CC32BAB
:10078000CB014B15CC2B4B1DC82BCB01CB15CC2B48
:100790004B1ECC2BCB014B15441DF32B461DE42BDC
:1007A000CC1CD52BCC014C15012C4C1DDA2BCC01CB
:1007B000CC15012CCC1DDF2BCC014C16012C4C1E72
:1007C000012CCC01CC14012C4C1DE92BCC014C1676
:1007D000012CCC1DEE2BCC014C16012C4C1E012CF7
:1007E000CC01CC14012CCC1CF82BCC014C15012CC9
:1007F0004C1DFD2BCC01CC15012C4C1E012CCC0129
:100800004C15C41D292CC61D1A2CCD1C0B2CCD013A
:100810004D155F13372C4D1D102CCD01CD15372CE8
:10082000CD1D152CCD014D16372C4D1E372CCD016D
:10083000CD14372C4D1D1F2CCD014D16372CCD1D41
:10084000242CCD014D16372C4D1E372CCD01CD1447
:10085000372CCD1C2E2CCD014D15372C4D1D332C96
:10086000CD01CD15372C4D1E372CCD014D155F1BFD
:10087000602C441E602C461E512CCE1C422CCE01F6
:100880004E156E2C4E1D472CCE01CE156E2CCE1D56
:100890004C2CCE014E166E2C4E1E6E2CCE01CE145C
:1008A0006E2C4E1D562CCE014E166E2CCE1D5B2C82
:1008B000CE014E166E2C4E1E6E2CCE01CE146E2C1A
:1008C000CE1C652CCE014E156E2C4E1D6A2CCE0111
:1008D000CE156E2C4E1E6E2CCE014E15C41E952CC0
:1008E000C61E862CCF1C772CCF014F15A32C4F1D75
:1008F0007C2CCF01CF15A32CCF1D812CCF014F16FF
:10090000A32C4F1EA32CCF01CF14A32C4F1D8B2C37
:10091000CF014F16A32CCF1D902CCF014F16A32C27
:100920004F1EA32CCF01CF14A32CCF1C9A2CCF0188
:100930004F15A32C4F1D9F2CCF01CF15A32C4F1E5D
:10094000A32CCF014F15441FCA2C461FBB2CD01C13
:10095000AC2CD0015015D82C501DB12CD001D01585
:10096000D82CD01DB62CD0015016D82C501ED82C07
:10097000D001D014D82C501DC02CD0015016D82C2A
:10098000D01DC52CD0015016D82C501ED82CD0010B
:10099000D014D82CD01CCF2CD0015015D82C501DE1
:1009A000D42CD001D015D82C501ED82CD0015015E5
:1009B000C41FFF2CC61FF02CD11CE12CD1015115F6
:1009C0000D2D511DE62CD101D1150D2DD11DEB2C76
:1009D000D10151160D2D511E0D2DD101D1140D2D0A
:1009E000511DF52CD10151160D2DD11DFA2CD1011F
:1009F00051160D2D511E0D2DD101D1140D2DD11CCF
:100A0000042DD10151150D2D511D092DD101D115E7
:100A10000D2D511E0D2DD1015115DF18372D451FFC
:100A2000372D471F282DD21C192DD2015215DF1347
:100A3000452D521D1E2DD201D215452DD21D232D1F
:100A4000D2015216452D521E452DD201D214452DEC
:100A5000521D2D2DD2015216452DD21D322DD201FF
:100A60005216452D521E452DD201D214452DD21CB1
:100A70003C2DD2015215452D521D412DD201D215CA
:100A8000452D521E452DD2015215DF18702DDF1B4A
:100A9000702DC51F702DC71F612DD31C522DD30182
:100AA00053157E2D531D572DD301D3157E2DD31DE8
:100AB0005C2DD30153167E2D531E7E2DD301D314EE
:100AC0007E2D531D662DD30153167E2DD31D6B2D08
:100AD000D30153167E2D531E7E2DD301D3147E2DAC
:100AE000D31C752DD30153157E2D531D7A2DD301A3
:100AF000D3157E2D531E7E2DD3015315D6214008CC
:100B0000C4004108C5005F18DF145F1CDF104808EF
:100B1000C9000C304A05031D05120C304B05031D9E
:100B200085120C304C05031D05100C304D05031DBE
:100B300085100C304E05031D87100C304F05031D2A
:100B400007110C305005031D07100C305105031D13
:100B500087120C305205031D07120C305305031D7C
:100B6000871149080E020318E12D12304A05031DB2
:100B7000051612304B05031D851612304C05031D5A
:100B8000051412304D05031D851412304E05031D4A
:100B9000871412304F05031D071512305005031D31
:100BA000071412305105031D871612305205031D1C
:100BB000071612305305031D8715FF30480203192D
:100BC00008008F08031D0800972049080E02031C27
:100BD000E12D18304A05031D051206304A05031D94
:100BE000051618304B05031D851206304B05031DF5
:100BF000851618304C05031D051006304C05031DE5
:100C0000051418304D05031D851006304D05031DD4
:100C1000851418304E05031D871006304E05031D40
:100C2000871418304F05031D071106304F05031DAB
:100C3000071518305005031D071006305005031D19
:100C4000071418305105031D871206305105031D86
:100C5000871618305205031D071206305205031D72
:100C6000071618305305031D871106305305031D61
:040C700087150800DC
:084000000500030002000600A8
:02400E00CC33B1
:10420000010078007A007C007E007B0079007F004E
:104210007D007A0078007E007C007D007F00FF003A
:104220008100F200F600FA00FE00F200F600FA004B
:10423000FE00F200F600FA00FE00F200F600FF00B9
:10424000FF00050005000500050009000900090040
:1042500009000D000D000D000D0011001100FF0000
:104260000000FF00FF00FF00FF00FF00FF00FF0055
:10427000FF00FF00FF00FF00FF00FF00FF00FF0046
:10428000FF00FF00FF00FF00FF00FF00FF00FF0036
:10429000FF00FF00FF00FF00FF00FF00FF00FF0026
:1042A000FF00FF00FF00FF00FF00FF00FF00FF0016
:1042B000FF00FF00FF00FF00FF00FF00FF00FF0006
:1042C000FF00FF00FF00FF00FF00FF00FF00FF00F6
:1042D000FF00FF00FF00FF00FF00FF00FF00FF00E6
:1042E000FF00FF00FF00FF00FF00FF00FF00FF00D6
:1042F000FF00FF00FF00FF00FF00FF00FF00DD00E8
:00000001FF
